:100000005EC1000078C1000076C1000074C100002C
:1000100072C1000070C100006EC100006CC1000020
:100020006AC1000068C1000066C100000C947D0D2B
:1000300062C1000060C100005EC100005CC1000040
:100040005AC1000058C1000056C1000054C1000050
:1000500052C1000050C100004EC100004CC1000060
:100060004AC1000048C1000046C1000044C1000070
:1000700042C10000DB02E002EB02F502FB020103D9
:100080002E033A033F0344035303580363037F03E0
:1000900092039803A003A603AC03B6030604260448
:1000A0003C044B04F404FB0404050B0515051B0577
:1000B0001E0525051E0525051E0525053F054605CA
:1000C0004F0556055F05650568056F0568056F05F1
:1000D00068056F054D0650065306560671067106F3
:1000E000710671065F06590665066B0662065C06B8
:1000F00068066E064A0E6D0E580F6D0E580FB40E40
:10010000D60E580F290F3B0F2203690062006D00C5
:100110002D00630061007000730065006E007300C5
:1001200065002D007500730062000000220354007A
:100130006F006D00200057006F006E0067002D00FB
:1001400043006F0072006E0061006C006C000000E4
:100150000403090409025400030100A0FA09040081
:1001600000010301010009211101000122250007FE
:1001700005810308000A09040100010300000009C9
:1001800021110100012220000705830308000A094C
:10019000040200010300000009211101000122BE38
:1001A000000705820319000A120110010000002057
:1001B000810402000100010200010600FF0901A103
:1001C000010902150025FF7508950881020903152C
:1001D0000025FF750895089102C005010906A101D7
:1001E00005081901290315002501950375019102E0
:1001F000950175059101050719E029E7150025010D
:10020000950875018102050719002931150025019E
:100210009532750181029501750181010507193338
:10022000299B1500250195697501810295017501CC
:1002300081010507199D29A415002501950875015F
:100240008102050119812983150025019503750196
:100250008102050C19B029B8150025019509750111
:100260008102050C09CD09E209E909EA0A8A010AB5
:1002700092010A94010A21020A23020A24020A2591
:10028000020A27020A2A0215002501950D7501812F
:1002900002950175028101C005010906A1017501E0
:1002A00095088101950175088101950575019101F8
:1002B000950175039101950675088101C00011240F
:1002C0001FBECFEFD4E0DEBFCDBF11E0A0E0B1E0B4
:1002D000ECE0F4E202C005900D92AC35B107D9F71D
:1002E00013E0ACE5B1E001C01D92A138B107E1F720
:1002F00090D00C94041284CE2AC310C380E291E003
:100300000E94C11080E191E00E94C11080E091E064
:100310000E94C110E2EEF0E0808184608083089545
:1003200080E291E00E948B0F80E191E00E948B0FB0
:1003300080E091E00C948B0F80912E0190912F0121
:10034000009729F0019790932F0180932E018091BF
:100350001E0190911F01009729F0019790931F01B2
:1003600080931E0180910E0190910F01009729F05A
:10037000019790930F0180930E01F7C20F931F9383
:10038000CF93DF93FC01C901E80121E0E032F207DD
:1003900011F412D405C021E0E031F20721F498D124
:1003A00088E090E005C066817781B9D489E190E06A
:1003B0009983888380E0DF91CF911F910F910895F9
:1003C000AC01C90121E04032520709F49EC54051F9
:1003D000514009F4E3C09CC584B7877F84BF88E19E
:1003E0000FB6F89480936000109260000FBE90E00A
:1003F00080E80FB6F89480936100909361000FBE7F
:100400000E945C0A0E948E0A0E94920A469A0C94EC
:100410006E0DE2DF7894BFD32DD7A4D7A4D38FE19C
:100420009EE40197F1F700C000000E947C0A8091D1
:10043000730390917403019609F42AD66CD58091C8
:100440007803882321F080917803853041F48091EE
:100450007603882321F0E4D681110E941A0B80E2F2
:1004600091E00E94D41080E191E00E94D41080E0DD
:1004700091E00E94D4100E94710FE0CF292F332702
:1004800023303105C9F064F42130310581F0223088
:10049000310509F043C084E590E024E531E042C035
:1004A00021323105F1F02232310541F137C082E1CC
:1004B00090E028EA31E036C099278130910541F07B
:1004C0008230910541F0892B49F5E0E5F1E005C066
:1004D000ECE2F1E002C0E8E0F1E0849190E09F01FD
:1004E00021C06330D8F4E62FF0E0EE0FFF1FE25C8E
:1004F000FE4F2081318189E090E014C0633070F4B8
:1005000070E0FB01EE0FFF1FE85CFE4F20813181A0
:10051000FB01EB5CFE4F808190E004C080E090E046
:1005200020E030E0FA01318320830895EF92FF92BA
:100530000F931F93CF93DF938C0191E0EE24E3940C
:10054000F12C461720F1A62FB0E0AA0FBB1FAA0F6F
:10055000BB1F20E030E0E801C90FD11DF901EA0F0F
:10056000FB1FE157FE4F808183304CF08881F701FB
:10057000022E01C0EE0F0A94EAF7E82BE8832F5F02
:100580003F4F2430310551F76F5F9F5FDACFDF9126
:10059000CF911F910F91FF90EF900895DC01EC91A6
:1005A0004E2F50E04D30510508F091C0FA01E65C45
:1005B000FF4F0C94A81111968C91809332010895ED
:1005C00011962C91119712968C9190E0982F882774
:1005D000820F911D72C711968C91882309F477C000
:1005E000E0913301F0913401099411968C918823A4
:1005F00009F46DC077C711968C91882309F467C000
:1006000047C513964C91139712969C911297119689
:10061000EC918E2F8F73873108F059C0943008F019
:1006200056C0E295E695E695E370E150E33040F47C
:10063000F0E0EE0FFF1FEC5BFE4F2081318102C026
:1006400026E532E0E82FF0E0EE0FFF1FEE0FFF1F70
:10065000E90FF11DE20FF31F4083089512968C916C
:1006600012971196EC91E83090F5F0E0E25FFC4FC4
:100670008083089511968C91882349F173C6119651
:100680008C91882321F18CC613968C911397129626
:100690009C91129711962C9120938D0190938C012F
:1006A00080938E0154C111968C91882381F049C2A8
:1006B00011968D919D91AC918093EB019093EC01FB
:1006C000A093ED01089511968C918111CBC50895E9
:1006D000CF93DF93DC0188E0FD0111928A95E9F761
:1006E000E0913201EC934E2F50E0FA013197EB305C
:1006F000F10508F0DAC0E95BFF4F0C94A81184E023
:1007000011968C93119798E012969C93129797E10B
:1007100013969C93139714968C93149781E01596D7
:100720008C93C3C046E060E0CD0100DF83E005C0EC
:100730004DE067E0CD01FADE84E080933201B5C080
:1007400044E16EE0CD01F2DE85E0F7CF47E165E1FF
:10075000CD01ECDE82E0F1CF9091730380917403C0
:1007600011969C93119712968C939FC0809187014C
:1007700090918601282F2295220F220F207C292B71
:1007800011962C931197C0913001D091310112969E
:10079000492F50E0440F551F440F551F20E030E013
:1007A000F901E40FF51FEC0FFD1F60816D932F5FC2
:1007B0003F4F24303105A1F79F5F973119F0909397
:1007C000860173C0109286018F5F843019F0809388
:1007D000870102C01092870180918701813061F00A
:1007E00040F0823081F0833009F05FC082EB92E00C
:1007F00005C086E592E002C086E193E09093310166
:100800008093300152C08AEF91E0F8CF809185014A
:1008100011968C931197E82FF0E0EE0FFF1FEE0F6B
:10082000FF1FE25FFC4F408151816281738112960C
:100830004D935D936D937C9315978F5F823019F084
:100840008093850132C0109285012FC0E6E5F1E06A
:1008500080E090E022E0280F31910196ED01C80F71
:10086000D91F3883332321F08630910599F727E08B
:10087000A20FB11D1C9219C080918D0111968C930D
:10088000119780918C0112968C93129780918E0112
:1008900013968C930AC02091EB013091EC014091AA
:1008A000ED0111962D933D934C93DF91CF910895D7
:1008B00090918801811103C091FD05C002C091FF94
:1008C00002C092FD10C0292F2170882331F096605C
:1008D0009093880181E0822708959D7F9460909392
:1008E0008801822F089580E008958823A1F08091E7
:1008F0008D018D3028F48B3040F4893020F4089538
:100900008F3028F0089581E003C082E001C083E0C9
:100910008093720308951092720308952498259885
:10092000269827982C982D982E982F9810928A0107
:1009300010928901809188018B7F8093880180913A
:100940008D01823019F4249A259A269A0895E6DFBB
:1009500080918D01813029F038F083508C3020F463
:100960002D9A269A279A2F9A089580918A018F3F6F
:1009700019F08F5F80938A0180918D01813021F081
:10098000C8F083508C30B0F490918A0180918C0132
:10099000981302C02E98089580918901882351F000
:1009A00020918E01921730F010928A01815080932D
:1009B00089012E9A0895809189018F5F8093890122
:1009C00008951F93CF93DF93162FE0918D014E2F43
:1009D00050E0FA013397EC30F10508F03CC0EC012F
:1009E000EE5AFF4F0C94A81183B185FB882780F93C
:1009F00091E0892702C083B180725ADF882359F1C0
:100A0000C10FD11D89E30FC083B185FB882780F911
:100A100091E0892702C083B180724ADF8823D9F030
:100A2000C10FD11D83E58A8316C01D9914C088812A
:100A30008E5F888310C01D99FACF0DC083B185FBEE
:100A4000882780F991E0892702C083B18072DF9105
:100A5000CF911F914ACFDF91CF911F910895CF93EE
:100A6000DF93E0918D014E2F50E0FA013397EC3087
:100A7000F105D0F5EC01E25AFF4F0C94A81183B1B7
:100A800085FB882780F991E0892702C083B18072B5
:100A90000FDF882349F188858260888725C083B16C
:100AA00085FB882780F991E0892702C083B1807295
:100AB000FFDE8823C9F08B8588608B8715C01D9960
:100AC00013C08881826088830FC01D99FACF0CC043
:100AD00083B185FB882780F991E0892702C083B123
:100AE0008072DF91CF9101CFDF91CF9108959091E6
:100AF0008D01953028F49330B0F4923021F00895B0
:100B00009730B8F0089580FF02C02D9A01C02D984B
:100B100081FF02C02E9A01C02E9882FF02C02C9A3B
:100B200008952C98089581FF06C080918801816006
:100B300005C080FDFACF809188018E7F8093880167
:100B4000089560918D018AE791E00E94F211609111
:100B50008C018BE791E00E94F21160918E018CE78D
:100B600091E00C94F2118AE791E00E94DB118F3042
:100B700018F480938D0102C010928D018BE791E0F3
:100B80000E94DB1180938C018CE791E00E94DB11C5
:100B900080938E0108958CE5EFE8F1E0DF011D926E
:100BA0008A95E9F78CE0EEEEF1E0DF011D928A957F
:100BB000E9F71092720308956F927F929F92AF921D
:100BC000BF92CF92DF92EF92FF920F931F93CF933A
:100BD000DF93EC0101D48150833048F4E82FF0E03A
:100BE000EE0FFF1FE65BFE4F4081518102C046E5DC
:100BF00052E000E010E060E0CC24C394D12CF3E09C
:100C0000BF2EA2E0AA2E99249394A62F20E030E0D4
:100C1000C80195958795FC01E251FE4F7F01702F29
:100C20007170663008F064C0F7018081E82FF0E051
:100C3000772351F0C9010496360102C0660C771C77
:100C40008A95E2F7C30107C0C601022E02C0880FD1
:100C5000991F0A94E2F78E239F23892B09F441C040
:100C6000FA01E20FF31FE081E430D8F180E38E0F48
:100C70008330B8F16F5FCE018A0F911DDC011296AF
:100C8000EC938E2F90E0FC01E85DF109E031F10575
:100C900040F5E659FF4F0C94A8111092720321C041
:100CA000909272031EC0A09272031BC0B092720396
:100CB00018C088818E5F14C08881805E11C08881D1
:100CC0008F5F0EC08881805F0BC088818C5F08C0F9
:100CD0008881805C05C08881885F02C088818058D7
:100CE00088832F5F3F4F2430310511F0A62F99CF15
:100CF0000F5F1F4F4C5F5F4F0731110509F085CF24
:100D0000CE01DF91CF911F910F91FF90EF90DF9077
:100D1000CF90BF90AF909F907F906F9052CE2F92C8
:100D20003F924F925F926F927F928F929F92AF927B
:100D3000BF92CF92DF92EF92FF920F931F93CF93C8
:100D4000DF9300D000D0CDB7DEB75C014B0144D3B8
:100D50008150833048F4E82FF0E0EE0FFF1FE65B90
:100D6000FE4F8081918102C086E592E07C01412C9A
:100D7000512C66246394712C3324339442E0242E46
:100D800000E010E0C20195958795FC01E251FE4F0D
:100D90006F01242D21702983F601808190E0298143
:100DA000222359F098012C5F3F4FA30102C0440F4A
:100DB000551F2A95E2F79A0107C09301002E02C041
:100DC000220F331F0A94E2F782239323892B09F41D
:100DD00073C0F701E00FF11F80818B3D31F188F482
:100DE000833D38F4803D08F067C0833008F464C068
:100DF0003CC0893DA1F0B0F4883DB9F51092720372
:100E00005BC0853E38F4823E18F5803E09F1813E94
:100E100081F02BC0853E69F0883ED0F026C030922C
:100E200072034AC02092720347C053E0509372038A
:100E300043C0F401208130E090E2980F02C0359564
:100E400027959A95E2F720FD03C08C83B4DD8C8151
:100E5000805E930102C0220F331F8A95E2F7C90119
:100E6000F5019081892B808327C0482F46954695B0
:100E7000469550E08770F401E40FF51F218130E0C2
:100E8000082E02C0359527950A94E2F720FD07C089
:100E90004A835B838C838FDD8C815B814A81FA017D
:100EA000EA0DFB1D930102C0220F331F8A95E2F762
:100EB000C9019181892B81830F5F1F4F0430110578
:100EC00009F06ACF3FEF431A530A44E0E40EF11CE5
:100ED00057E14516510409F053CFC5010F900F900B
:100EE0000F900F90DF91CF911F910F91FF90EF9096
:100EF000DF90CF90BF90AF909F908F907F906F903A
:100F00005F904F903F902F90AACDFC018081EFCD54
:100F1000FC018081ECCD4F925F927F928F929F92E5
:100F2000AF92BF92CF92DF92EF92FF920F931F93F7
:100F3000CF93DF9300D000D0CDB7DEB78CE0EEEEDC
:100F4000F1E0DF011D928A95E9F77FE8E72E71E075
:100F5000F72E00E010E0AA24A394E5E0BE2EDD24E5
:100F6000D394F8ECCF2E902EE02FE695E695E695FB
:100F7000F0E0E551FE4F808190E0202F277002C005
:100F8000959587952A95E2F780FD65C04698802F54
:100F9000D1D2469A19821A821B821C828A2D8A9586
:100FA000F1F71899A9821999AA821A99AB821B990B
:100FB000AC82AE014F5F5F4F2701D70120E030E0E8
:100FC000C8019595879582519E4FE92DE1709E2E1F
:100FD000722EFA016191AF01F201662319F060816E
:100FE000615002C060816F5F6083BD018C9087FE9D
:100FF00002C01C9204C0F5E0F8150CF4BC921196E6
:10100000FB0160816330B4F0FC018080992051F0D5
:10101000B9016C5F7F4FFD2D01C0FF0F6A95EAF7A4
:101020006F2F05C06D2D01C0660F7A94EAF768290D
:10103000FC0160832F5F3F4FFFEF4F1A5F0A2430A0
:10104000310531F646986ED2469A0631110519F0EF
:101050008C2D8A95F1F70F5F1F4F64E0E60EF11CAF
:101060000731110509F07FCF0F900F900F900F906F
:10107000DF91CF911F910F91FF90EF90DF90CF9074
:10108000BF90AF909F908F907F905F904F9008950A
:10109000AF92BF92CF92DF92EF92FF920F931F9386
:1010A000CF93DF9346E552E027E1B12CD12C80E0CD
:1010B00090E0FA01E80FF91F3081313021F0323031
:1010C00019F4D39401C0B39401968430910589F743
:1010D00021504C5F5F4F2111EACFC0E0D0E00FEF0D
:1010E0001FE0E12CF12CC8018E199F098230910577
:1010F000C0F1EC01D695C795CE0DDF1DCE01DDD137
:101100008FE891E00197F1F700C0000070E2C72E70
:1011100002DFCA94E9F72FE831E066E572E040E0CB
:1011200080E090E0F901E80FF91F508153303CF066
:10113000FB01E80FF91F5081543008F04F5F019612
:101140008430910579F72C5F3F4F6C5F7F4F91E0C2
:101150002B3E390729F74D1510F08E01C4CF7E01C3
:10116000C2CF8E01EE24EA945FE0F52EC12CD12C83
:1011700097012C193D0922303105C0F1E901D695BE
:10118000C795CC0DDD1DCE0198D18FE891E0019778
:10119000F1F700C0000040E2A42EBDDEAA94E9F7FA
:1011A0008FE891E066E572E040E020E030E0FC018D
:1011B000E20FF31F508153303CF0FB01E20FF31FAD
:1011C0005081513009F44F5F2F5F3F4F243031057C
:1011D00071F704966C5F7F4F21E08B3E920729F7F1
:1011E0004B1510F07E01C4CF6E01C2CFC8018C1B1D
:1011F0009D0B24E0969587952A95E1F76FE070E0C6
:101200000E9497118C0F9D1F58D1DF91CF911F9194
:101210000F91FF90EF90DF90CF90BF90AF9097CB62
:1012200026E532E04FE851E080E090E0FA01E80F77
:10123000F91F6081633034F0F901E80FF91F608114
:10124000643070F401968430910581F72C5F3F4F34
:101250004C5F5F4F82E0223B380731F780E0089512
:1012600081E0089543E050E06DE771E08BEE91E09E
:101270000C94E31143E050E06DE771E08BEE91E0F8
:101280000E94CB118091EB018F3F71F48091EC01B2
:101290008F3F51F48091ED018F3F31F41092EB01BB
:1012A0001092EC011092ED010895AF92BF92CF928F
:1012B000DF92EF92FF920F931F93CF93DF93EB0197
:1012C0005C012CE5A20EB11C6C01F4E0CF0ED11C28
:1012D0007E018C010F5F1F4F0E94DB118F3F09F4CD
:1012E00080E0F70181937F01C8010C151D0589F786
:1012F00024960A151B0541F7DF91CF911F910F919D
:10130000FF90EF90DF90CF90BF90AF900895AF9295
:10131000BF92CF92DF92FF920F931F93CF93DF93F1
:101320008C01EB0187E1F82E6E0184E0C80ED11C20
:10133000C80169915C012FEFA21AB20A0E94F21152
:10134000C501CC15DD05A9F70C5F1F4FFA9461F7B5
:10135000DF91CF911F910F91FF90DF90CF90BF90C1
:10136000AF90089510928B0148E050E062E771E081
:101370008EE093E00E94CB1166E572E082E090E09F
:1013800094DF66E173E08EE590E08FDF6AEF71E055
:101390008AEB90E08ADF62EB72E086E191E085CF34
:1013A00048E050E062E771E08EE093E00E94E311D4
:1013B00066E572E082E090E0AADF66E173E08EE528
:1013C00090E0A5DF6AEF71E08AEB90E0A0DF62EBCE
:1013D00072E086E191E09BCFEF92FF921F93CF9353
:1013E000DF9380917203E0918B01E150E33040F490
:1013F000F0E0EE0FFF1FE05BFE4F4081518102C025
:1014000046E552E060E070E090E0C1E0D0E0FB0132
:10141000F595E795E251FE4FA081B0E020E030E085
:10142000162F1170112351F0F90134967E0102C07C
:10143000EE0CFF1CEA95E2F7F70107C0FE01022E51
:1014400002C0EE0FFF1F0A94E2F7EA23FB23EF2B03
:1014500079F0FA01E20FF31FE081E13D31F0E23D66
:1014600031F0E03D29F4916003C0926001C09460C6
:101470002F5F3F4F24303105A9F66F5F7F4F4C5FE0
:101480005F4F6731710519F6992371F0EEE0F3E0D3
:1014900038E03E0F2191422F42954F70491302C010
:1014A000822F8F703E13F6CF80938B01DF91CF9107
:1014B0001F91FF90EF9008955BC0CF93DF9300D012
:1014C000CDB7DEB780937303909374039F709983B5
:1014D0008A8362E0CE0101967FD00F900F90DF915A
:1014E000CF9108956091730380E090E07BD7609185
:1014F000740381E090E076C7CF93DF9381E090E0C2
:101500005AD7C82FD0E0DC2FCC2780E090E053D70B
:101510009E01282BC901DF91CF91CFCF3C9A3D9AF4
:101520003E9A08954598449888E1459A4598815097
:10153000E1F7089545984498449A459A4598449807
:1015400090E0981721F0459A45989F5FFACF08954B
:10155000882321F05098489BFECF0895509A5898C0
:101560000895882311F051980895519A5998089533
:10157000509A519A81E0F5DF81E0EACF80E0F1DF17
:1015800000C080E0E5DF00C081E00895489B03C013
:10159000509A589808955098489BFECF0895CF933D
:1015A000DF93D82FC8E08D2F881F8827881FD9DFA9
:1015B000EDDF00C0EBDFDD0F00C0C150A1F7519897
:1015C000E5DF499905C000C0E1DF519A00C0C1E0E4
:1015D0008C2FDF91CF910895EF92FF920F931F937D
:1015E000CF93DF93C82FE92ED62FC8DF811102C019
:1015F00080E019C080ECD3DF8823D1F3FC2E0C2FC0
:101600001E2DC0E0802F8F198D1738F4F8018191BD
:101610008F01C5DFC82F8111F5CF81E099DF000070
:1016200081E09FDF8C2FDF91CF911F910F91FF9071
:10163000EF90089584E089BD86E089BD09B400FE7D
:10164000FDCF8091D8008F7D8093D8008091E000FD
:1016500082608093E0008091E00081FDFCCF0895DE
:10166000CF92DF92EF92FF920F931F93CF93DF936E
:10167000EC018B017A01C9D1811133C0E114F1046D
:1016800039F0F70180819181081B190BC80FD91F10
:10169000C12CD12C0115110519F18091E80085FDAF
:1016A00016C08091E8008E778093E8001AD4E11488
:1016B000F10449F0F70180819181C80ED91ED182D1
:1016C000C08285E00EC0A1D1882321F30AC0899190
:1016D0008093F10001501109FFEFCF1ADF0ADACF32
:1016E00080E0DF91CF911F910F91FF90EF90DF90FD
:1016F000CF90089520917F033091800326173707FC
:1017000048F06115710539F42091E8002E77209397
:10171000E80001C0B90140E06115710581F1209137
:1017200078032223E9F12530E9F12091E80023FD37
:1017300035C02091E80022FD2BC02091E80020FF59
:10174000EBCF2091F20030E0FC01CF016115710573
:1017500059F02032310540F481918093F1006150BD
:1017600071092F5F3F4FF1CF41E02032310509F081
:1017700040E02091E8002E772093E800CDCF411182
:10178000CECF06C080917803882351F0853051F088
:101790008091E80082FFF6CF80E0089581E008950F
:1017A00082E0089583E008956115710529F4209180
:1017B000E8002B772093E800FC016115710521F109
:1017C00080917803882341F1853041F18091E800D0
:1017D00083FD20C08091E80082FFEFCF8091F2006E
:1017E000882331F08091F100819361507109B1F744
:1017F0008091E8008B778093E800DFCF80917803B9
:10180000882351F0853051F08091E80080FFF6CFB9
:1018100080E0089581E0089582E0089583E00895CE
:1018200020917F03309180032617370748F0611518
:10183000710539F42091E8002E772093E80001C06B
:10184000B901FC0120E06115710569F1809178030F
:101850008823D1F18530D1F18091E80083FD32C039
:101860008091E80082FD28C08091E80080FFEBCFE6
:101870008091F20090E06115710559F08032910578
:1018800040F424912093F100319661507109019642
:10189000F2CF21E0809709F020E08091E8008E7778
:1018A0008093E800D0CF2111D1CF06C0809178037A
:1018B000882351F0853051F08091E80082FFF6CF07
:1018C00080E0089581E0089582E0089583E008951E
:1018D000982F953058F59093E900981739F070914A
:1018E000EC002091ED005091F00003C0242F762FE2
:1018F00050E021FF19C03091EB003E7F3093EB00A8
:101900003091ED003D7F3093ED003091EB00316080
:101910003093EB007093EC002093ED005093F000B7
:101920002091EE0027FF07C09F5FD3CF8F70809379
:10193000E90081E0089580E00895EF92FF920F930F
:101940001F93CF93DF93E62EEC018C010C5F1F4FAA
:10195000F12CFE1499F19881992359F1F801208115
:1019600069817A8131973081892F8F70853010F0AD
:1019700080E025C0223010F442E001C046E0E8E0FB
:10198000F0E020E0E617F70720F42F5FEE0FFF1FCF
:10199000F9CF2295207F422B232F2295220F220F51
:1019A000207C991F9927991F622F692B91DF88232B
:1019B000F9F2F39425960B5F1F4FCBCF81E0DF91B7
:1019C000CF911F910F91FF90EF900895809179032F
:1019D00087FF11C08091E80082FD05C080917803E7
:1019E0008111F8CF11C08091E8008B770BC08091F6
:1019F0007803882349F08091E80080FFF8CF809138
:101A0000E8008E778093E80008952091E4003091FB
:101A1000E50095E64091EC00842F817040FF22C0E4
:101A20008091E80080FD1CC080917803882391F0AC
:101A3000853091F08091EB0085FD10C04091E4006D
:101A40005091E5004217530729F39A01915011F77D
:101A500084E0089582E0089583E0089581E0089588
:101A600080E008954091E80042FFDECF08953FD026
:101A700041D08091D8008F778093D8008091D80092
:101A800080688093D8008091D8008F7D8093D800A3
:101A900084E089BD86E089BD09B400FEFDCF1092C7
:101AA0007803109275031092760342E260E080E0C2
:101AB0000FDF8091E1008E7F8093E1008091E20052
:101AC00081608093E2008091E20088608093E20070
:101AD0008091E0008E7F8093E0000895E3E6F0E0DF
:101AE00080818E7F808381E080937703C0CF1092C6
:101AF000E20008951092E10008951F920F920FB630
:101B00000F9211242F933F934F935F936F937F9383
:101B10008F939F93AF93BF93EF93FF938091E100D7
:101B200082FF0BC08091E20082FF07C08091E1003C
:101B30008B7F8093E1000E949C018091E10080FFF7
:101B400018C08091E20080FF14C08091E2008E7F77
:101B50008093E2008091E20080618093E2008091B6
:101B6000D80080628093D80019BC109278030E943C
:101B70007D018091E10084FF2EC08091E20084FF0E
:101B80002AC084E089BD86E089BD09B400FEFDCF8E
:101B90008091D8008F7D8093D8008091E1008F7E66
:101BA0008093E1008091E2008F7E8093E20080913B
:101BB000E20081608093E20080917503811106C08C
:101BC0008091E30087FD02C081E001C084E0809342
:101BD00078030E947C018091E10083FF22C0809104
:101BE000E20083FF1EC08091E100877F8093E100C7
:101BF00082E080937803109275038091E1008E7FDC
:101C00008093E1008091E2008E7F8093E2008091DA
:101C1000E20080618093E20042E260E080E058DE12
:101C20005FD1FF91EF91BF91AF919F918F917F9184
:101C30006F915F914F913F912F910F900FBE0F9039
:101C40001F9018951F93CF93DF93CDB7DEB7AA9758
:101C50000FB6F894DEBF0FBECDBFE9E7F3E088E032
:101C60008E0F9091F10091938E13FBCF0E94900103
:101C70008091E80083FF1CC18091790390917A03E1
:101C8000492F50E04A30510508F012C1FA01E658D8
:101C9000FF4F5EC3803881F0823809F009C180911E
:101CA0007D038F708093E9008091EB0085FB88278E
:101CB00080F91092E90007C080917603882311F023
:101CC00082E001C080E09091E800977F9093E80067
:101CD0008093F1001092F100C7C0282F2D7F09F0EA
:101CE000E7C0882319F0823061F0E2C080917B0365
:101CF000813009F0DDC0933009F080E080937603F5
:101D00002DC080917B03811129C080917D038F704C
:101D100009F4CEC08093E9009091EB0090FF1EC0C3
:101D200090917A03933021F48091EB00806214C08B
:101D30009091EB0090619093EB0021E030E0A901DD
:101D400002C0440F551F8A95E2F74093EA001092B3
:101D5000EA008091EB0088608093EB001092E9002C
:101D60008091E800877F83C08111A2C010917B031E
:101D70001F778091E3008078812B8093E30080912E
:101D8000E800877F8093E80021DE8091E80080FFF3
:101D9000FCCF8091E30080688093E300111102C0C2
:101DA00082E001C083E08093780382C08058823053
:101DB00008F07EC080917B0390917C038C3D53E0C2
:101DC000950771F583E08A838AE289834FB7F89497
:101DD000DE01139620E03EE051E2E32FF0E0509365
:101DE0005700E49120FF03C0E295EF703F5FEF7072
:101DF0008E2F90E0EA3010F0C79601C0C0968D9308
:101E00009D932F5F243149F74FBF8091E800877F72
:101E10008093E8006AE270E0CE0101966BDC13C0AB
:101E2000AE014F5F5F4F60917D030E943E02BC0197
:101E3000009709F43DC09091E800977F9093E800E7
:101E400089819A81EDDC8091E8008B778093E800AE
:101E50002FC0803869F58091E800877F8093E80083
:101E6000809175038093F1008091E8008E778093D4
:101E7000E800ACDD1DC081111BC090917B03923046
:101E8000B8F48091E800877F8093E8009093750311
:101E90009DDD80917503811106C08091E30087FD6F
:101EA00002C081E001C084E0809378030E947E013B
:101EB0008091E80083FF0AC08091E800877F8093CB
:101EC000E8008091EB0080628093EB00AA960FB649
:101ED000F894DEBF0FBECDBFDF91CF911F91089563
:101EE0000895CF9380917803882399F0C091E900F9
:101EF000CF709091EC00892F817090FD80E8C82B05
:101F00001092E9008091E80083FD9CDECF70C093C1
:101F1000E900CF9108956F927F928F929F92AF9236
:101F2000BF92CF92DF92EF92FF920F931F93CF93C6
:101F3000DF9300D01F92CDB7DEB77C01CDB6DEB601
:101F40008091E80083FF06C1F701808190E0209135
:101F50007D0330917E032817390709F0FBC080917B
:101F60007A03833009F49DC030F4813071F08230FF
:101F700009F4D4C0EFC08A3009F4B8C08B3009F43A
:101F8000A1C0893009F0E6C04EC080917903813A42
:101F900009F0E0C08DB69EB61A82198280917B034B
:101FA00010917C038B83F7018085482F50E08DB71B
:101FB0009EB7841B950B0FB6F8949EBF0FBE8DBFC6
:101FC000EDB7FEB731965F0160E070E0CF01DCD184
:101FD0004FEF410F8E010F5F1F4F9501BE016D5FE7
:101FE0007F4FC7010E94BE01F7018681978100974C
:101FF00021F0408550E0B501BED11092E9008091FA
:10200000E800877F8093E80069817A81C50172DBEF
:102010008091E8008B778093E8000FB6F8949EBE1D
:102020000FBE8DBE97C080917903813209F092C0B6
:10203000ADB6BEB600917F031091800370907B0314
:1020400060907C038DB79EB7801B910B0FB6F89400
:102050009EBF0FBE8DBFEDB7FEB731964F01809189
:10206000E800877F8093E800B801CF019DDB809175
:10207000E8008E778093E80021E0711001C020E035
:1020800030E0021B130B280D391D4FEF460D672D55
:10209000C7010E94E0010FB6F894BEBE0FBEADBEF0
:1020A00059C080917903813A09F054C08091E800C9
:1020B000877F8093E8008091E80080FFFCCFF701E4
:1020C000818540C080917903813209F043C08091BD
:1020D000E800877F8093E80079DC90917B0381E0C2
:1020E000911101C080E0F701818734C080917903AC
:1020F000813281F58091E800877F8093E80066DC7B
:1021000080917B0390917C03882736E09695879594
:102110003A95E1F7F701958784871CC08091790390
:10212000813AC1F48091E800877F8093E800809134
:10213000E80080FFFCCFF70184859585969587950B
:10214000969587958093F1008091E8008E77809333
:10215000E8003CDC0FB6F894DEBE0FBECDBE0F909B
:102160000F900F90DF91CF911F910F91FF90EF9003
:10217000DF90CF90BF90AF909F908F907F906F90A7
:102180000895FC01399627E0DF011D922A95E9F7B1
:1021900021E0FC01218724EF31E03587248723E00B
:1021A000248361E00196C9CB4F925F926F927F9238
:1021B0008F929F92AF92BF92CF92DF92EF92FF9257
:1021C0000F931F93CF93DF9300D01F92CDB7DEB74D
:1021D0007C01ADB6BEB680917803843009F08EC024
:1021E0008091E4009091E500F7012285338528175E
:1021F000390709F483C081818F708093E900809151
:10220000E80085FF7BC08DB69EB6408550E08DB757
:102210009EB7841B950B0FB6F8949EBF0FBE8DBF63
:10222000EDB7FEB731966F011B821A82198260E00A
:1022300070E0CF01A9D08E010F5F1F4F960140E0E3
:10224000BE016D5F7F4FC7010E94BE01482EF7019E
:1022500084859585892B51F091E080E0268537852E
:10226000232B09F090E0092F182F02C000E010E0A6
:10227000F701668077806114710489F049815A8181
:10228000B301C6016BD055245394892B09F4512C0A
:10229000F701408550E0B601C3016DD001C0512C5B
:1022A00089819A81892BF1F0411004C0511002C03C
:1022B000012BC1F0F70184859585978786878181F9
:1022C0008F708093E9008B8181118093F100698187
:1022D0007A8140E050E0C601C3D98091E8008E7752
:1022E0008093E8008091E4009091E500F7019387E6
:1022F00082870FB6F8949EBE0FBE8DBE0FB6F894BF
:10230000BEBE0FBEADBE0F900F900F90DF91CF916C
:102310001F910F91FF90EF90DF90CF90BF90AF9003
:102320009F908F907F906F905F904F9008950024C2
:10233000552704C0080E591F880F991F009729F0D0
:1023400076956795B8F37105B9F7802D952F0895A7
:10235000EE0FFF1F0590F491E02D0994FB01DC01C5
:1023600004C08D910190801921F441505040C8F76C
:10237000881B990B0895FB01DC0102C001900D92AE
:1023800041505040D8F70895DC0101C06D93415091
:102390005040E0F70895DC01CB01FC01F999FECF34
:1023A00006C0F2BDE1BDF89A319600B40D924150DD
:1023B0005040B8F70895F999FECF92BD81BDF89AC3
:1023C000992780B50895DC01A40FB51F41505040F6
:1023D00040F0CB01840F951F2E9105D04150504005
:1023E000D8F70895262FF999FECF92BD81BDF89AAE
:1023F000019700B4021639F01FBA20BD0FB6F89449
:0C240000FA9AF99A0FBE0895F894FFCFE5
:10240C000282190000015C011900000000000000AC
:10241C0001830800000175010800000000000000A5
:10242C000081080000017D01080000000000000090
:10243C0056020200182520BE9802BA01DA01660184
:10244C007F0198011603FA01B2021603FA01B202D7
:0C245C001603FA01B202302E372E3000B9
:00000001FF
